:020000000F28C7
:10000800FE00030EF1000408F2000A08F300831250
:100018007F08F400722BD82BF02AF22AF42AF62A49
:10002800F82AFA2AFC2AFE2A002B022B042B062B7C
:10003800082B0A2B0C2B0E2B102B122B142B162BE8
:10004800182B1A2B1C2B202B222B242B262B282B4E
:100058002A2B2C2B2E2B612A652A692A8A2A8A2A7E
:100068008A2A8A2A8A2A6A2A6E2A722A762A7A2A60
:060078007E2A822A862A7E
:10020000FF1B0A2983137F1883170008840A031928
:10021000FF0A08007F087F398A000408840A03194E
:10022000FF0A82002634A6348634A8346A34603447
:10023000AA348A34A83486348334A33460348634B0
:10024000A8348A34AD348D34AD348F34AF348D342A
:10025000AD3468346034A0348D34AA348D34AD3478
:100260008D34AD348E34A0348E34AE3491348F342A
:10027000AF346A348034A8348A34AD348D34AD342C
:100280008A34AA348834A8348634A6340034263418
:1002900082348234A23447344E348B34AA348934C5
:1002A00053346E348B34AA34893453346E348B34E3
:1002B000AA348B34493482348234A23447344E34E5
:1002C0008B34AA34893453346E348B34AA34893451
:1002D00053346E348B34AA348B3449346234A234B0
:1002E00044348E348B348A3489348734A734893447
:1002F000AA346934003430346D348D34AB34AD34C9
:10030000AF34AD34AB34AA348D34AD34AA346D344B
:100310008D34AB34AD34AA34A834A534A634483473
:10032000A834A634A534A334A534A634A834AA34FA
:1003300068346834A834AA34AB34AA34A834A63458
:10034000A534A334A534A33481348134A134A33437
:100350008534863463344834003413348434A5340B
:10036000603480348734A834603480348434A534D5
:10037000A034C0348734A834A034C0348D348B34D6
:10038000C0348534A834A034C0348B344A34A0340B
:10039000C034AA3488348534A3348534003411340D
:1003A00079347934763477349634773474346034ED
:1003B00079347934763497349634803474346034B4
:1003C00071347134743472349134723499348D349C
:1003D0008F347134913491348034913474340034D6
:1003E0002334913491349134913491349134A5343F
:1003F000AA34AD34B1349034903490349034903485
:100400009034A634AA34AD34B0346F348D348A3489
:100410008D346D344A34CA34CD34D13496340034FA
:10042000263468348A34AA34A834A034A8348D34ED
:100430008834863468348F34AF34A834A034A83478
:1004400090348F348A3488348F349434A834A6346A
:10045000A034A63483348A344834003420349534AC
:10046000913495349A3476346034933490349334A0
:100470009734753493349134603491348E347334BA
:100480006E346034933491347534733400341034E2
:10049000CD34CE34CF34CE34CD3400341034813426
:1004A0008034813400341034D93400348312A600EF
:1004B0008B1307168230831681008312A401A40ACD
:1004C0008F2A5330A90082308D2A4730A90082300C
:1004D0008D2A8A2AF030A90081308D2A1030A90097
:1004E00082308D2A7B30A90081308D2A4730A900C7
:1004F00081308D2A2E30A90082308D2ACF30A9007C
:1005000081308D2A1230A90081308D2AAD30A900AA
:1005100081308D2A4E30A9008230AA009A2A2608FE
:1005200084001030040203188A2A00308A002F3019
:10053000040782002A08FF00290884000021F50032
:100540007508A7000130A9070318AA0AA3012A0801
:10055000FF00290884000021003803196A2B2A08AB
:10056000FF00290884000021F5007508A80001306B
:10057000A9070318AA0ACE2A4030C72A2030C72A62
:100580001030C72A0830C72A0430C72A0230F500C5
:100590007508A000EB2AA001A00AEB2A2808E03980
:1005A000F500F6017608003A0319D72ACB2A750818
:1005B000203A0319BC2A603A0319BE2A203A0319CB
:1005C000C02AE03A0319C22A203A0319C42A603A21
:1005D0000319C62ACB2A2008F5007508A200392B7A
:1005E000EE301D2BE1301D2BD4301D2BC8301D2BC0
:1005F000BD301D2BB2301D2BA8301D2B9E301D2B66
:1006000096301D2B8D301D2B85301D2B7E301D2BE4
:1006100076301D2B70301D2B69301D2B63301D2B48
:100620005E301D2B59301D2B54301D2B4F301D2B90
:100630004A301D2B46301D2B423083169200352B3D
:10064000FC302F2BEE302F2BE1302F2BD4302F2BE3
:10065000C8302F2BBD302F2BB2302F2BA830831654
:1006600092000530362B83169201073083129200D8
:10067000502B28081F39F500F6017608003A0319B7
:10068000422B332B7508FF3E031C332B84001F3095
:1006900004020318332B00308A0010300407820054
:1006A0002708F5007508A1007D3081008B168316A0
:1006B0001208F5000310750C831293000C3095009E
:1006C0008B1783122308031D672B6400612B8B1388
:1006D0009501A62AA4018430831681008312071293
:1006E0008B1708000B1DA12B0B112408013A031DC9
:1006F0008A2B7D3081000130A202031DA12B20082E
:10070000F0007008A2000130A102031DA12BA3017B
:10071000A30AA12B063081000130AB02AB08031DF8
:10072000992B7D30F0007008AB000430F0007008A9
:10073000A50025080319A02B0130A5020716A12B3F
:1007400007127408FF0073088A0072088400710E93
:100750008300FE0E7E0E09008B0107308312990084
:1007600083169101831295018316850183128501F9
:100770000F30831687000F30831287008430831672
:1007800081007D30F70077088312AB00A5010630A9
:1007900081008B168B17A40183120718D12B003010
:1007A000562283128718D62B023056226400CC2B97
:1007B000A001A101A201A301A401A5018301AC2B09
:02400E00E9F3D4
:00000001FF
